:1000000012C0189518951895189518951895189563
:10001000189513C118951895189518951895189551
:100020001895189518958FE58DBFC0E4E0E44E2E25
:1000300084E08EBFD4E0F4E05F2EEEEFF3E0A0E6C4
:10004000B0E088278D933197E9F766248FEF87BB5F
:1000500081E088BB80E084BB8FEF85BB8FEF81BBE5
:1000600080E082BBE1D383E083BF89B7816089BF31
:10007000789480E080937200809160008064809327
:100080006000E2E0F0E0A5E7B0E091E0B6D30091D7
:100090007500043609F006C080916000806180938D
:1000A000600005C0809160008F7E80936000E3E077
:1000B000F0E0A6E6B0E091E0A0D3E4E0F0E0A7E64F
:1000C000B0E091E09AD300916600073110F009F09A
:1000D00001C003C088E080936600009167000B3385
:1000E00010F009F001C003C080E080936700002792
:1000F000A0E6B0E08C9187FB0EF401E041E004172C
:1001000009F007C0809160008F7780936000E3D092
:10011000CBD10027A0E6B0E08C9186FB0EF401E085
:1001200041E0041709F086C0809160008F7B8093C6
:100130006000A0E6B0E08C9185FB882780F980956F
:1001400080FBA0E6B0E08C9185F98C930091720061
:10015000003009F02BC06DD312EA82D312E080D3B5
:1001600068D313EA7DD39BD3AAE6B0E01C9397D360
:10017000A9E6B0E01C9391D3A8E6B0E01C9367D346
:10018000AAE6B0E09C910FD3A5E6B0E08C93A9E677
:10019000B0E09C9108D3A4E6B0E08C93A8E6B0E070
:1001A0009C9101D3A3E6B0E08C9330C0013009F0FC
:1001B0000FC0A3E7B0E08C918F5F8C930091730028
:1001C000083009F004C080D280E0809372001EC025
:1001D000023009F01BC0A4E7B0E08C918F5F8C93D4
:1001E00000917400083009F011C0E3E0F0E0A6E6E9
:1001F000B0E091E07BE7F0D2E4E0F0E0A7E6B0E029
:1002000091E07BE7E9D280E0809372000091760074
:10021000003010F009F001C00CC0C0988091760049
:1002200081508093760000917600003009F001C083
:10023000C09A76D25CCFF894FFCF0F921F922F9284
:100240003F924F925F927F92AF92BF920F931F9314
:100250002F933F934F935F936F937F938F939F93CE
:10026000AF93BF93CF93DF93EF93FF938FB78F93AA
:1002700080916000806880936000A2E6B0E08C917D
:100280008F5F8C93009162000A3F08F408C080E001
:1002900080936200809160008064809360008F9101
:1002A0008FBFFF91EF91DF91CF91BF91AF919F9160
:1002B0008F917F916F915F914F913F912F911F91FE
:1002C0000F91BF90AF907F905F904F903F902F9095
:1002D0001F900F901895ABE6B0E08C918F5F8C93D8
:1002E00000916B00083009F003C080E080936B0040
:1002F00000917200003009F012C0A0E6B0E08C91CD
:1003000085FBA8E3B0E08C9181F98C938091630028
:1003100080936D008091640080936E0019C001305D
:1003200009F00AC0C19A8091630080936D008091AA
:10033000640080936E000CC0023009F009C0C198BF
:100340008091660080936D008091670080936E00BD
:1003500000916B00003009F012C000916D004AE07E
:1003600053D2ACE6B0E00C9300916C00003009F081
:1003700003C08AE080936C003DD0C59A3AC001303A
:1003800009F002C0C59835C0023009F00AC00091DA
:100390006D004AE039D2ACE6B0E08C932BD0C49A21
:1003A00028C0033009F002C0C49823C0043009F00B
:1003B0000AC000916E004AE027D2ACE6B0E00C9390
:1003C00019D0C39A16C0053009F002C0C39811C0F5
:1003D000063009F00AC000916E004AE015D2ACE682
:1003E000B0E08C9307D0C29A04C0073009F001C076
:1003F000C298089500916C00003009F005C0C698BD
:10040000C79880E882BB4FC0013009F005C0C6988C
:10041000C79880E482BB47C0023009F005C0C69887
:10042000C79880E282BB3FC0033009F005C0C69880
:10043000C79A80E082BB37C0043009F005C0C69A75
:10044000C79880E082BB2FC0053009F005C0C69870
:10045000C79880E182BB27C0063009F005C0C69866
:10046000C79888E082BB1FC0073009F005C0C69856
:10047000C79884E082BB17C0083009F005C0C69851
:10048000C79882E082BB0FC0093009F005C0C6984A
:10049000C79881E082BB07C00A3009F004C0C69843
:1004A000C79880E082BB0895A1E7B0E083B38C9346
:1004B000A1E7B0E08C91806F8C93009171000F3FA9
:1004C00081E009F480E08F93409171000091700009
:1004D000041781E009F080E09F918923882309F4C3
:1004E000EBC0AFE6B0E08C918F5F8C9300916F0012
:1004F000003509F0E0C080E080936F00009170004B
:10050000073F09F03AC000917200003009F013C0B3
:10051000809160008F7E8093600080E08093750002
:10052000E2E0F0E0A5E7B0E091E07BE755D182E0C2
:100530008093760021C0013009F00EC080916300E5
:10054000815080936300009163000F3F09F003C066
:1005500087E18093630010C0023009F00DC08091E4
:100560006600815080936600009166000F3F09F09D
:1005700003C087E18093660098C00B3F09F02BC051
:1005800000917200003009F004C081E08093720095
:1005900021C0013009F00EC0A3E6B0E08C918F5F5E
:1005A0008C9300916300083109F003C080E08093D0
:1005B000630010C0023009F00DC0A6E6B0E08C91D7
:1005C0008F5F8C9300916600083109F003C080E0D2
:1005D000809366006AC00D3F09F03AC00091720036
:1005E000003009F013C0809160008061809360004A
:1005F00084E680937500E2E0F0E0A5E7B0E091E0EA
:100600007BE7EAD083E08093760021C0013009F0D7
:100610000EC080916400815080936400009164005A
:100620000F3F09F003C08BE38093640010C00230D9
:1006300009F00DC0809167008150809367000091A0
:1006400067000F3F09F003C08BE3809367002DC064
:100650000E3F09F02AC000917200003009F004C07A
:1006600082E08093720021C0013009F00EC0A4E640
:10067000B0E08C918F5F8C93009164000C3309F093
:1006800003C080E08093640010C0023009F00DC008
:10069000A7E6B0E08C918F5F8C93009167000C33DC
:1006A00009F003C080E08093670080E080937300CE
:1006B00080E08093740007C0809171008093700087
:1006C0008CE380936F000895A3E6B0E08C9165D031
:1006D000A8E6B0E08C93A4E6B0E08C915ED0A9E6E9
:1006E000B0E08C9380E080936A00A3D012EAB8D087
:1006F00010E0B6D018E0B4D0AAD09BD012EAB0D0A7
:1007000012E0AED0AAE6B0E01C91AAD0A9E6B0E013
:100710001C91A6D0A8E6B0E01C91A2D098D0089574
:100720000027A0E6B0E08C9184FB0EF401E041E0EC
:10073000041709F026C04091660000916300041779
:1007400081E009F080E08F934091670000916400A0
:10075000041781E009F080E09F918923882309F440
:100760000AC0A0E6B0E08C9185FBA8E3B0E08C91D4
:1007700080F98C9306C000917600003009F001C02A
:10078000C09A0895982F82958F70805D8D939F7089
:10079000905D9D9388278C9308954AE0082F34D06C
:1007A0000295802B0895892F8F70905110F0865FED
:1007B000FCCF08953197F1F70895689462F8089591
:1007C000E89462F80895E199FECFEEBBFFBB319645
:1007D000089591E001C092E07B3751F47FB7F8941F
:1007E000F2DF8D918DBBE29AE19A9A95C9F77FBFAE
:1007F0007727089591E001C092E0E5DFE09A8DB39C
:100800008D939A95D1F70895FF93881BF9E0001F07
:10081000FA9511F4FF910895881F841B18F4840F32
:100820008894F5CF0894F3CFAC98AD98A498A59888
:100830000895A59AA49803D0A59801D0A49AEF93FF
:10084000FF93E6E0F0E0B6DFFF91EF910895A59AFF
:10085000A49AF5DFA5989D9BFECFF1DFA498EFCF7A
:100860000894111F01C0110F69F0A59A18F4000037
:10087000A49802C0A49A00C0E2DFA5989D9BFECF79
:10088000DEDFF1CFA59AA498DADFA5989D9BFECF75
:10089000E8949C99689462F8D2CF089401C0889437
:1008A000331F11E0A59AA498CADFA5989D9BFECF9F
:1008B000C6DF88949C990894111FA0F7A59A3795D4
:1008C00010F4A49801C0A49ABADFA5989D9BFECF0E
:0408D000B6DF0895F2
:00000001FF
